:020000020000FC
:10000000F8940FED0DBF0FEF01BB03E001BB0FEF45
:1000100007BB0DD01ED019D007D038E729D024D087
:1000200006D038E725D0F6CF9098919A0895909A07
:10003000919808950FEF08BB0895C09A0895C19A4A
:100040000895C29A0895C39A0895C49A0895C59AC6
:10005000089500E008BB0895C0980895C1980895D8
:10006000C2980895C3980895C4980895C5980895AE
:10007000112422241A94F1F72A94E1F73A95D1F742
:020080000895E1
:00000001FF
